:020000040800F2
:10000000E00700204D17000805030008070300085B
:100010000B0300080F030008130300080000000092
:1000200000000000000000000000000017030008AE
:1000300019030008000000001B0300081D0300084E
:100040006717000867170008671700086717000898
:100050006717000867170008671700086717000888
:100060006717000867170008671700086717000878
:100070006717000867170008671700086717000868
:100080006717000867170008671700086717000858
:100090006717000867170008671700086717000848
:1000A0006717000867170008671700086717000838
:1000B0006717000867170008671700086717000828
:1000C0006717000867170008671700086717000818
:1000D00067170008332000084B200008892000081B
:1000E00067170008671700086717000800F002F894
:1000F00000F03FF80AA090E8000C82448344AAF183
:100100000107DA4501D100F034F8AFF2090EBAE880
:100110000F0013F0010F18BFFB1A43F0010318473B
:1001200088210000A8210000103A24BF78C878C1B7
:10013000FAD8520724BF30C830C144BF04680C60ED
:10014000704700000023002400250026103A28BF35
:1001500078C1FBD8520728BF30C148BF0B60704739
:10016000732902F03E80002070471FB51FBD10B5F7
:1001700010BD02F069F81146FFF7F7FF00F04CF8E8
:1001800002F087F803B4FFF7F2FF03BC01F014FE9E
:1001900010B552A001F094FF4FF4967001F0D9FD14
:1001A00050A1514801F0F5FF044650A001F088FF2E
:1001B0004FF4967001F0CDFD4AA14B4801F0E9FFE4
:1001C000044601F019FBC4B901204A4908604FF404
:1001D000967001F0BEFD4FF4967001F0BAFD4FF439
:1001E000967001F0B6FD4FF4967001F0B2FD00205C
:1001F0004149C1F8800101F0FFFA38A001F060FF29
:100200004FF4967001F0A5FD01F0F6FA35A13648DD
:1002100001F0BFFF044610BD86B001F05DFD01F0A6
:10022000C5FD01F0B3FA4FF4E13001F0EFFD4FF4FA
:10023000E13001F03AFE40F27121072001F0CAFAE4
:1002400000BF01F02AFD0028FBD1FFF7A1FF01F05C
:10025000EAFA01F09EFB3FE004A905A801F0F1FCD9
:100260009DF814000A2190FBF1F03030C0B28DF8F7
:1002700004009DF8140090FBF1F201FB12003030F5
:10028000C0B28DF805009DF8100090FBF1F0303001
:10029000C0B28DF806009DF8100090FBF1F201FB52
:1002A00012003030C0B28DF8070000208DF8080031
:1002B00001A912A001F078FB4FF4FA7001F049FD9A
:1002C00001F0B0FB0E48006808B9012000E00020F2
:1002D0000B49086001F090FABEE7000041540D0A96
:1002E000000000004F4B0000B70000204154653073
:1002F0000D0A00008001214200002142340000006C
:1003000080812142704700BFFEE700BFFEE700BFCB
:10031000FEE700BFFEE77047704770477047000078
:1003200010B500F03DFE012000F0BFFE00BF21200F
:1003300000F079FE0028FAD0102000F099F9022090
:1003400000F082F9002000F0D0FE002000F0DFFE77
:100350004FF4806000F0D2FE4FF46011002000F0F6
:10036000A7FE012000F0B0FE00BF392000F05BFEC8
:100370000028FAD0022000F0AAFE00BF00F0B0FE74
:100380000828FBD101211D2000F078FF10BD0CB51D
:100390000020019000906C48006840F480306A4969
:1003A000086000BF6848006800F4003000900198C1
:1003B000401C0190009818B90198B0F5A06FF1D1D8
:1003C0006148006800F4003010B10120009001E0A5
:1003D000002000900098012843D15C48006840F05C
:1003E00010005A4908600846006820F003000860C1
:1003F0000846006840F002000860534840685249CF
:1004000048600846406848600846406840F480609C
:1004100048600846406820F47C1048600846406800
:1004200040F4E81048600846006840F080700860BA
:1004300000BF4548006800F000700028F9D042482D
:10044000406820F00300404948600846406840F09A
:100450000200486000BF3C48406800F00C000828DB
:10046000F9D10CBD10B5FFF792FF10BD10B536489D
:10047000006840F00100344908600846406834498B
:1004800008403149486008460068324908402E4912
:1004900008600846006820F480200860084640682C
:1004A00020F4FE0048604FF41F008860FFF7DAFF79
:1004B0004FF000602849086010BD10B500210020F1
:1004C0000022214B5B6803F00C0121B1042906D006
:1004D000082928D107E0214B214C236027E01F4B3E
:1004E0001F4C236023E0184B5B6803F47010164B1D
:1004F0005B6803F48032022303EB904022B9194B6E
:100500004343174C23600DE00F4B5B6803F400334B
:1005100023B1144B4343124C236003E00F4B43437E
:100520000F4C236003E00D4B0D4C236000BF00BF58
:10053000054B5B68C3F303130B4CE15C084B1B6872
:10054000CB40074C236010BD001002400020024049
:100550000000FFF8FFFFF6FE08ED00E000127A0051
:100560000000002000093D00040000203149014343
:10057000314A1160704770B5002100230F22C47802
:1005800004B32D4C246804F4E064C4F5E064210A4B
:10059000C1F10403CA40447804FA03F1847814409A
:1005A00021430901254C0678A155047804F01F0564
:1005B0000124AC4005786D11AD0005F1E025C5F8CA
:1005C000004109E0047804F01F050124AC401C4DF3
:1005D0000678761145F8264070BD1A4A0A40024353
:1005E000154B1B1F1A60704739B1134A121D126850
:1005F0000243114B1B1D1A6006E00F4A121D1268C0
:1006000082430D4B1B1D1A607047042808D14FF020
:10061000E021096941F004014FF0E022116107E097
:100620004FF0E021096921F004014FF0E02211614F
:10063000704700000000FA050CED00E000E400E067
:1006400080E100E080FFFF1F01460020FE4A1068A5
:1006500000F03800084310607047FB49096821F03A
:100660000801F94A11601146096801431160704799
:10067000F549096821F01001F34A11601146096833
:10068000014311607047F148EF494860F048486005
:100690007047EE48EC494860ED4848607047EA48CA
:1006A000006940F08000E84908617047E648006949
:1006B00040F08000E449086170470420E249C968BD
:1006C00001F0010109B101200EE0DF49C96801F024
:1006D000040109B1022007E0DB49C96801F01001FB
:1006E00009B1032000E00420704700B5024604234E
:1006F000FFF7E3FF034603E0FFF7DFFF0346521E69
:10070000012B01D1002AF7D102B90523184600BDFB
:1007100030B5044604254FF43020FFF7E6FF0546C8
:10072000042D17D1C848006940F00200C64908618D
:1007300008464461006940F0400008614FF43020F1
:10074000FFF7D3FF0546C048006941F6FD71084038
:10075000BD490861284630BD10B504244FF430204F
:10076000FFF7C3FF0446042C16D1B748006940F0D8
:100770000400B54908610846006940F0400008617E
:100780004FF43020FFF7B1FF0446AF48006941F64F
:10079000FB710840AC490861204610BD00B5024617
:1007A0000423FFF78AFF034603E0FFF786FF0346B3
:1007B000521E012B01D1002AF7D102B90523184698
:1007C00000BD10B504244FF43020FFF7E7FF0446C6
:1007D000042C16D19C48006940F004009A49086135
:1007E0000846006940F0400008614FF43020FFF7F0
:1007F000D5FF04469448006941F6FB7108409249D0
:100800000861204610BD00208F49C96901F002012E
:1008100009B1012000E00020704730B5A52504246F
:10082000FFF7F1FF00B100254FF43020FFF75DFF27
:100830000446042C3AD185488349886084488860FE
:100840000846006940F0200008610846006940F051
:10085000400008614FF43020FFF747FF0446042CA6
:100860001BD17948006941F6DF710840764908617B
:100870000846006940F01000086176480580E002F3
:10088000FFF733FF0446052C10D06F48006941F68E
:10089000EF7108406C49086108E0052C06D06A48F1
:1008A000006941F6EF71084067490861204630BD94
:1008B00078B506460C46042500200090E802FFF7B4
:1008C00014FF0546042D24D15F48006940F0010063
:1008D0005D4908613480E802FFF707FF0546042DF3
:1008E00010D1B01C0090200C00990880E802FFF79E
:1008F000FCFE05465448006941F6FE710840524925
:10090000086106E05048006941F6FE7108404E4912
:100910000861284678BD70B504460D460426F002ED
:10092000FFF7E3FE0646042E11D14748006940F068
:100930000100454908612580F002FFF7D6FE064612
:100940004148006941F6FE7108403F490861304660
:1009500070BD70B505460E460424E002FFF7C5FEE3
:100960000446042C17D139483749886038488860D4
:100970000846006940F0100008612E80E002FFF791
:10098000B4FE0446052C06D02F48006941F6EF71ED
:1009900008402D490861204670BD2DE9F04304460A
:1009A0004FF6FF763746B046B1460425E443E6B23B
:1009B000C4F30727C4F307484FEA1469E802FFF7B6
:1009C00094FE0546042D49D120481F4988602048DF
:1009D00088600846006940F010000861FF2E06D0CC
:1009E0001C4808300680E802FFF77FFE0546042D0C
:1009F00008D1FF2F06D017480A300780E802FFF71A
:100A000074FE0546042D0AD1B8F1FF0F07D0114836
:100A10000C30A0F80080E802FFF767FE0546042DC1
:100A20000AD1B9F1FF0F07D00A480E30A0F80090A4
:100A3000E802FFF75AFE0546052D0FD0024800696F
:100A400041F6EF71084007E00020024023016745AE
:100A5000AB89EFCD00F8FF1F664908612846BDE865
:100A6000F08330B5054604244FF43020FFF73DFEF7
:100A70000446042C41D160485E4988605F48886024
:100A80000846006940F0200008610846006940F00F
:100A9000400008614FF43020FFF727FE0446042C85
:100AA00022D15448006941F6DF710840514908617C
:100AB0000846006940F0100008611DB1002050494F
:100AC000088002E0A5204E4908804FF43020FFF74F
:100AD0000CFE0446052C10D04648006941F6EF7123
:100AE00008404449086108E0052C06D041480069E7
:100AF00041F6DF7108403F490861204630BDF0B53E
:100B000005460E46174604243B483A4988603B4850
:100B10008860E002FFF7E9FD0446042C19D135484E
:100B2000006940F010003349086147F0F800304395
:100B300028433349891C0880E002FFF7D6FD0446AC
:100B4000052C06D02B48006941F6EF710840294971
:100B500008612046F0BD2748C069800870472548D5
:100B6000006A704700202349096801F0200109B19B
:100B7000012000E00020704729B11E4A126902439B
:100B80001C4B1A6104E01B4A12698243194B1A611B
:100B9000704701460020012908D1164AD26902F0A7
:100BA00001020AB1012008E0002006E0114AD268E3
:100BB0000A400AB1012000E0002070470D49C860DA
:100BC000704704200B49C96801F0010109B10120F7
:100BD0000EE00849C96801F0040109B1022007E0EC
:100BE0000449C96801F0100109B1032000E00420A4
:100BF000704700000020024023016745AB89EFCD1C
:100C000000F8FF1F10B50446CC48844208D10121EA
:100C1000042000F04DFB0021042000F049FB46E0D9
:100C2000C748844208D10121082000F041FB00217F
:100C3000082000F03DFB3AE0C248844208D101217F
:100C4000102000F035FB0021102000F031FB2EE0D9
:100C5000BD48844208D10121202000F029FB002159
:100C6000202000F025FB22E0B848844208D1012171
:100C7000402000F01DFB0021402000F019FB16E091
:100C8000B348844208D10121802000F011FB0021EB
:100C9000802000F00DFB0AE0AE48844207D101211C
:100CA000801500F005FB0021A01500F001FB10BD30
:100CB00010B50121084600F0FBFA0021012000F0E8
:100CC000F7FA10BD2DE9F04102460025002600206C
:100CD00000230024002791F803C00CF00F0591F8C1
:100CE00003C00CF0100CBCF1000F03D091F802C04F
:100CF0004CEA050591F800C0BCF1000F31D0146832
:100D000000202BE04FF0010C0CFA00F3B1F800C00A
:100D10000CEA03069E4220D183004FF00F0C0CFA20
:100D200003F7BC4305FA03FC4CEA040491F803C042
:100D3000BCF1280F06D14FF0010C0CFA00FCC2F8F0
:100D400014C00AE091F803C0BCF1480F05D14FF080
:100D5000010C0CFA00FCC2F810C0401C0828D1D3CA
:100D60001460B1F800C0BCF1FF0F34DD54680020FE
:100D70002EE000F1080C4FF0010808FA0CF3B1F86E
:100D800000C00CEA03069E4221D183004FF00F0CF5
:100D90000CFA03F7BC4305FA03FC4CEA040491F88F
:100DA00003C0BCF1280F05D100F1080C08FA0CF8BB
:100DB000C2F8148091F803C0BCF1480F07D100F1CC
:100DC000080C4FF0010808FA0CF8C2F81080401C1B
:100DD0000828CED35460BDE8F0814FF6FF71018042
:100DE000022181700421C17070470246002093687F
:100DF0000B400BB1012000E00020704701468868DD
:100E000080B2704702460020D3680B400BB101202E
:100E100000E0002070470146C86880B27047016159
:100E20007047416170470AB1016100E0416170475C
:100E3000C16070474FF480320A43826181618261F0
:100E400082698269704702460020434B18684FF65A
:100E50008073184040EA021008433F4B1860704707
:100E60003E49C8617047F0B50A46002300240021BE
:100E7000002500F00046B6F1004F02D1364EF16970
:100E800001E0354E7168C0F3034583B200F44016AB
:100E9000B6F5401F08D121F070612F4E766826F01C
:100EA00070662D4F7E6012E000F48016B6F5801F4C
:100EB00006D1032606FA05F4A14341F0706106E06D
:100EC000460D360103FA06F6B14341F0706122B1D6
:100ED000460D360103FA06F6314300F00046B6F13E
:100EE000004F02D11C4EF16101E01B4E7160F0BD5C
:100EF00030B500228B071C0F0F2303FA04F2164BA8
:100F000008338C1053F824309343134C08348D105D
:100F100044F8253023468C1053F824308C07240FD6
:100F200000FA04F423430C4C08348D1044F82530A7
:100F300030BD0A49DC3108607047000000080140FC
:100F4000000C014000100140001401400018014055
:100F5000001C014000200140000001400000204230
:100F60000E49086070470D49486070470B4988601A
:100F700070474AF6AA200949086070474CF6CC40F1
:100F800006490860704701460020044AD2680A40BA
:100F90000AB1012000E0002070470000003000404E
:100FA000DF48006840F00100DD49086008464068FD
:100FB000DC490840DA49486008460068DA490840D8
:100FC000D74908600846006820F480200860084679
:100FD000406820F4FE0048604FF41F0088607047AE
:100FE000CF49096821F48031CD4A11601146096862
:100FF00021F480211160B0F5803F03D0B0F5802F3F
:101000000ED106E0C649096841F48031C44A116036
:1010100007E0C349096841F4A021C14A116000E01A
:1010200000BF00BF704710B501460022002300201A
:101030004A11012A02D1BA4C236806E0022A02D1E1
:10104000B74C236A01E0B64C636A01F01F02012429
:1010500094401C400CB1012000E0002010BD38B5C8
:10106000002000900024002500BF3120FFF7DBFFA7
:1010700005460098401C00900098B0F5A06F01D084
:10108000002DF2D03120FFF7CEFF08B1012400E09F
:101090000024204638BD01460020A14A106820F0F7
:1010A000F80040EAC10010607047A049086070472E
:1010B000024600209A4B586820F47C1042EA010353
:1010C0001843974B58607047984908667047014627
:1010D0000020934A506820F0030008435060704796
:1010E0008F48406800F00C007047014600208C4A91
:1010F000506820F0F000084350607047014600201F
:10110000874A506820F4E060084350607047014609
:101110000020834A506820F4605040EAC1005060CB
:10112000704729B17E4A527A02437D4B5A7204E0DD
:101130007B4A527A82437A4B5A7270477B49D83144
:101140000860704701460020754A506820F440400E
:101150000843506070470021714A20321170704A74
:1011600082F82010012802D004280AD104E00121CD
:101170006B4A2032117005E00521694A2032117056
:1011800000E000BF00BF70476949086070476449CC
:10119000096A0143624A116270476549443908602F
:1011A000704730B500210022002400235C4D6D689B
:1011B00005F00C0121B1042905D0082923D105E04F
:1011C0005C4D056022E05B4D05601FE0544D6D688D
:1011D00005F47012524D6D6805F48034022505EB5C
:1011E00092421CB9544D554305600BE04C4D6D685F
:1011F00005F400351DB1504D5543056002E04D4DDD
:101200005543056002E04B4D056000BF00BF444DF3
:101210006D6805F0F0010909484D6B5C0568DD401B
:1012200045603F4D6D6805F4E061090A434D6B5C14
:101230004568DD4085603A4D6D6805F46051C90A26
:101240003E4D6B5C4568DD40C560354D6D6805F40D
:101250004041890B3A4D6B5CC568B5FBF3F5056100
:1012600030BD29B12E4A526902432D4B5A6104E028
:101270002B4A526982432A4B5A61704729B1284A46
:1012800092690243264B9A6104E0254A926982439F
:10129000234B9A61704729B1214AD2690243204BFE
:1012A000DA6104E01E4AD26982431D4BDA6170475D
:1012B00029B11B4AD2680243194BDA6004E0184A8C
:1012C000D2688243164BDA60704729B1144A12691A
:1012D0000243134B1A6104E0114A12698243104B16
:1012E0001A61704712494039086070470F49C86455
:1012F00070470B49C87170470948406A40F08070D8
:1013000007494862704701460020054A92680A4032
:101310000AB1012000E0002070470149887270473F
:10132000001002400000FFF8FFFFF6FE00004242FE
:101330008004424200127A0000093D00140000209F
:101340002400002010B50446FB48844209D1012145
:101350008803FFF7ADFF00214FF48040FFF7A8FF9F
:1013600032E0F648844209D101214804FFF7ADFF7D
:1013700000214FF40030FFF7A8FF25E0F048844239
:1013800009D101218804FFF7A0FF00214FF480203C
:10139000FFF79BFF18E0EB48844209D10121C80404
:1013A000FFF793FF00214FF40020FFF78EFF0BE0C3
:1013B000E548844208D101210805FFF786FF002196
:1013C0004FF48010FFF781FF10BD2DE9F04786B084
:1013D00005460E460024A24600BFA1460027B0895C
:1013E00000B100BF2F462C8A4CF6FF700440F088F5
:1013F00004432C82AC894EF6F3100440B088318946
:101400000843718908430443AC81AC8A4FF6FF401E
:101410000440B0890443AC8201A8FFF7C2FEC6486D
:10142000874202D1DDF810A001E0DDF80CA0A88908
:1014300000F4004040B10AEBCA0000EB0A1031682A
:101440004900B0FBF1F807E00AEBCA0000EB0A1014
:1014500031688900B0FBF1F86420B8FBF0F00401BA
:101460002009642101FB1089A88900F4004040B1E3
:10147000322000EBC900B0FBF1F000F0070004439C
:1014800008E0322000EB09106421B0FBF1F000F01D
:101490000F0004432C8106B0BDE8F0874FF41651CD
:1014A000016000218180C18001810C2141810021E6
:1014B0008181704710B502460020108A4FF2FF0369
:1014C00018400B884C8823438C882343CC882343C3
:1014D0001843108210BD0021018041808180C180AD
:1014E000704721B1828942F40052828104E08289EE
:1014F0004DF6FF731A4082817047F0B50346002411
:1015000000260025002040F66A17B94200D100BF2E
:101510001846C1F3421401F01F06012707FA06F529
:10152000012C01D10C3004E0022C01D1103000E07C
:1015300014301AB107682F43076002E00768AF4311
:101540000760F0BD1AB1838A0B43838202E0838A6D
:101550008B4383827047028A4FF6F0731A400282EF
:10156000028A0A430282704782894FF2FF731A404F
:10157000828182890A438281704721B1828942F047
:101580000202828104E082894FF6FD731A40828153
:101590007047028A4FF6DF731A400282028A0A43BA
:1015A0000282704721B1028A42F48042028204E042
:1015B000028A4BF6FF731A4002827047C1F3080299
:1015C0008280704701468888C0F30800704781898F
:1015D00041F0010181817047028BD2B20283028BFC
:1015E00042EA012202837047028B02F47F420283A7
:1015F000028B0A430283704721B1828A42F02002A3
:10160000828204E0828A4FF6DF731A40828270473A
:1016100021B1828A42F01002828204E0828A4FF66F
:10162000EF731A408282704721B1828A42F0080229
:10163000828204E0828A4FF6F7731A4082827047F2
:1016400021B1828942F40042828103E08289C2F39F
:101650000E028281704721B1828A42F40062828246
:1016600004E0828A4FF2FF731A4082827047828AB6
:101670004FF6FB731A408282828A0A438282704745
:1016800021B1828A42F00202828204E0828A4FF60D
:10169000FD731A408282704702460020B1F5007F38
:1016A00000D100BF13880B400BB1012000E00020E7
:1016B000704701F40072B2F5007F00D100BFCA4349
:1016C0000280704770B502460024002300250020E8
:1016D00040F66A16B14200D100BFC1F3421501F0D5
:1016E0001F03012606FA03F3012D02D19689334028
:1016F00006E0022D02D1168A334001E0968A33407B
:101700000C12012606FA04F41688344013B10CB109
:10171000012000E0002070BD10B50022002340F63B
:101720006A14A14200D100BF0A1201249440A3B25E
:10173000DC43048010BD000000380140004400403C
:1017400000480040004C00400050004009488047DD
:1017500009480047FEE7FEE7FEE7FEE7FEE7FEE793
:10176000FEE7FEE7FEE7FEE704480549054A064BAB
:10177000704700006D040008ED000008E001002043
:10178000E0070020E0030020E003002008B501216D
:101790000C20FFF773FD0120ADF8000010208DF83C
:1017A000030003208DF8020069460848FFF78AFA13
:1017B0000120ADF8000010208DF8030003208DF803
:1017C000020069460248FFF77DFA08BD000C01409F
:1017D0000008014070B505460C4645F25550FFF72C
:1017E000BFFB2846FFF7BFFB2046FFF7BFFBFFF715
:1017F000C0FBFFF7C3FB70BD10B5FFF7BAFB10BD10
:1018000010B58F4800F0F3FB002404E000208C4961
:101810000855601CC4B2642CF8DB002089490870AC
:10182000FFF7EAFF10BD10B587A000F049FC4FF4A8
:10183000967000F08EFA86A1814800F0AAFC8549D6
:101840000860FFF7DDFF0EE0FFF7DAFF7EA000F093
:1018500037FC4FF4967000F07CFA7DA1784800F0D8
:1018600098FC7C4908607B4800680028ECD07AA08E
:1018700000F026FC4FF4967000F06BFA79A000F0AF
:101880001FFC4FF4967000F064FA79A16C4800F0E8
:1018900080FC70490860FFF7B3FF0EE0FFF7B0FF70
:1018A00070A000F00DFC4FF4967000F052FA70A199
:1018B000634800F06EFC67490860664800680028CD
:1018C000ECD06CA000F0FCFB4FF4967000F041FAF5
:1018D0005FA15B4800F05DFC5E490860FFF790FF88
:1018E00068A000F0EDFB4FF4967000F032FA68A1AA
:1018F000534800F04EFC57490860FFF781FF0EE0A7
:10190000FFF77EFF5FA000F0DBFB4FF4967000F066
:1019100020FA5FA14A4800F03CFC4E4908604D485F
:1019200000680028ECD05DA000F0CAFB4FF4967070
:1019300000F00FFA5CA1424800F02BFC454908601A
:101940000846006810B308460068007A3038096815
:10195000C979303901EB810100EB4100544908702D
:1019600008460078632804D03A480068C0793038C7
:1019700040B906E000204E4981F872004DA000F009
:1019800047FBF7E701204A4981F87200FFF738FF6B
:1019900010BD10B54EA000F093FB4FF4967000F010
:1019A000D8F9FFF72DFF10BD70B504460D462A4645
:1019B000214654A000F084FB4FF4967000F0C9F962
:1019C00008E055A11E4800F0E4FB224908606420AD
:1019D00000F0BFF91F4800680028F2D0184800F056
:1019E00006FB00201749087070BD70B504460D460F
:1019F0002A4621464AA000F063FB4FF4967000F09F
:101A0000A8F908E044A10E4800F0C3FB11490860A2
:101A1000642000F09EF90F4800680028F2D0FFF71C
:101A2000EFFE70BD10B544A1054800F0B2FB0949B6
:101A300008600846006808B1FFF7E2FE10BD00002C
:101A4000B70000204000002041540D0A00000000B3
:101A50004F4B00002800002041542B4346554E3D7B
:101A6000310D0A0041542B43494D490D0A00000035
:101A70003436300041542B43474154543D310D0A14
:101A80000000000041542B43474154543F0D0A00CD
:101A90002B43474154543A203100000041542B431A
:101AA0004553510D0A0000002B43455351000000DF
:101AB00044000020D0C5BAC5CBD1CBF7CAA7B0DC53
:101AC000A3ACC7EBB2E9BFB4D4ADD2F2210D0A008A
:101AD00041542B51494F50454E3D312C302C22550D
:101AE0004450222C2234372E39322E3134362E32C5
:101AF0003130222C393939392C313233342C310DF3
:101B00000A00000041542B514953454E443D302CAE
:101B100025732C25730D0A0053454E44204F4B006E
:101B200041542B514953454E4445583D302C257363
:101B30002C25730D0A0000002B2B51495552433AB6
:101B40000000000010B56048006820F0F0005E4919
:101B500008600846006840F03000086000205B49DB
:101B60000860142000F0F5F801205949C1F88401FB
:101B70001E2000F0CAF810BD10B5002452480068BD
:101B800020F0F000504908600846006840F08000EE
:101B9000086004E0601CC4B2012000F0B6F84B48B5
:101BA0008038006808B1642CF4DB642C01DB012070
:101BB00010BD002404E0601CC4B2012000F0A5F8B0
:101BC00042488038006808B9642CF4DB642C01DBDF
:101BD0000120EDE70020EBE710B5002404E0601CD5
:101BE000C4B2012000F091F838488038006808B18C
:101BF000642CF4DB002404E0601CC4B2012000F07B
:101C000084F832488038006808B9642CF4DB282056
:101C100000F07BF82D488038006808B1012010BD25
:101C20000020FCE770B50024002506E06006040EE5
:101C3000FFF7D2FF0443681CC5B2082DF6DB20462F
:101C400070BD7CB505460E46FFF77CFFFFF794FF9D
:101C5000F8B9002405E0FFF7E5FF0DF80400601C6B
:101C6000C4B2052CF7DB9DF800009DF80110084474
:101C70009DF8021008449DF8031008449DF80410D4
:101C8000884208D19DF8000030709DF8020028704D
:101C900001E001207CBD0020FCE710B50D48806903
:101CA00040F008000B4988610748006820F0704048
:101CB000054908600846006840F030000860FFF7FA
:101CC00041FFFFF759FF10BD000C01408481214204
:101CD000008021420010024010B56FF00400FEF7B2
:101CE00094FC2E4800682E49B0FBF1F02D49087095
:101CF0000846007800EB4001C1EBC0104FF6FF71C1
:101D000001EAC0002849088010BD0146254A127822
:101D10004A434FF0E0235A6100229A611A46126941
:101D200042F001021A6100BF4FF0E022106900F09A
:101D300001021AB100F48032002AF5D04FF0E022FF
:101D4000126922F001024FF0E0231A6100229A6129
:101D500070470146144A12884A434FF0E0235A6103
:101D600000229A611A46126942F001021A6100BF0C
:101D70004FF0E022106900F001021AB100F4803245
:101D8000002AF5D04FF0E022126922F001024FF054
:101D9000E0231A6100229A617047000000000020D1
:101DA00000127A00320000203400002010B54FF4F9
:101DB000A060FEF7DBFB10BD00BF704700BFB84A54
:101DC000128802F04002002AF9D0C2B2B44B1B1DA7
:101DD0001A80704710B5044600BF8021B148FFF754
:101DE0005BFC0028F9D02146AE48FFF7E7FB10BDA9
:101DF00010B5044600BF8021A948FFF74DFC00281C
:101E0000F9D02146A648FFF7D9FB10BD10B586B022
:101E10000446012144F20400FFF730FAA148FFF71D
:101E200091FA4FF40070ADF8140003208DF81600FD
:101E300018208DF8170005A99B48FEF743FF4FF4C3
:101E40008060ADF8140048208DF8170005A9964869
:101E5000FEF738FF25208DF8000003208DF80100E3
:101E60008DF8020001208DF803006846FEF783FB21
:101E700001940020ADF80800ADF80A00ADF80C00A0
:101E8000ADF810000C20ADF80E0001A98548FFF751
:101E90009CFA012240F225518248FFF72EFB0121D6
:101EA0008048FFF71EFB06B010BD10B586B0044693
:101EB00001210420FFF7E2F901214804FFF7EBF9C3
:101EC0007748FFF73FFA0420ADF8140003208DF89F
:101ED000160018208DF8170005A97348FEF7F2FECA
:101EE0000820ADF8140004208DF8170005A96E48ED
:101EF000FEF7E8FE26208DF8000000208DF8010096
:101F000001208DF802008DF803006846FEF733FBD0
:101F100001940020ADF80800ADF80A00ADF80C00FF
:101F2000ADF810000C20ADF80E0001A95C48FFF7D9
:101F30004CFA012240F225515948FFF7DEFA0121FF
:101F40005748FFF7CEFA06B010BD10B586B004466C
:101F500001210820FFF792F901218804FFF79BF97E
:101F60005248FFF7EFF94FF48060ADF814000320FA
:101F70008DF8160018208DF8170005A94C48FEF7BB
:101F8000A1FE4FF40060ADF8140004208DF8170096
:101F900005A94748FEF796FE27208DF8000000208F
:101FA0008DF8010001208DF802008DF803006846CD
:101FB000FEF7E1FA01940020ADF80800ADF80A0040
:101FC000ADF80C00ADF810000C20ADF80E0001A922
:101FD0003648FFF7FAF9012240F225513348FFF75E
:101FE0008CFA01213148FFF77CFA06B010BD0BE0F6
:101FF00000BF2C49098801F040010029F9D001787F
:10200000284A121D1180401C01780029F0D1704728
:102010000BE000BF2549098801F040010029F9D0F3
:102020000178224A121D1180401C01780029F0D14C
:10203000704710B540F225511A48FFF743FB18B11D
:102040001848FFF7BFFAC4B210BD10B540F22551D1
:102050001348FFF737FBB0B11148FFF7B3FAC4B22A
:102060000F48FFF7AFFAC1B2124802780078401C5F
:10207000104B18701048815418460078632802DD10
:1020800000201946087010BD10B540F225510748D0
:10209000FFF718FB18B10548FFF794FAC4B210BD5A
:1020A0000044004000380140000801400048004062
:1020B000000C014040000020B700002070470000E5
:1020C0000FB4044910B503AA029800F08FF810BCB1
:1020D0005DF814FB3C0000202DE9F0410E4604465B
:1020E000002020622046E168884730B3252805D0CB
:1020F000D4E901219047206A401CF2E7E1682046BC
:1021000000278847050018D0A5F14100192802D8FA
:1021100020354FF400673246294620462760FEF7F7
:102120001FF840B1012804D0F61D26F00706083636
:10213000D8E7361DD6E72846DAE7206ABDE8F08101
:1021400070B50C460546012A05D02878800600D5D2
:10215000EA69002302E0012305E05B1C934202D2FE
:10216000E05C0028F9D1A869E618C01AA861286ABD
:10217000184428622846AFF3008004E0D5E9012125
:1021800014F8010B9047B442F8D32846AFF300800F
:1021900070BD30B505460B462A4613F8014B12F8C0
:1021A000010B08B1A042F8D01CB1002802D06D1C70
:1021B000F1E7284630BD704770477047704710B54B
:1021C000436913B1AFF3008001E0FFF7B9FF0120CD
:1021D00010BD127800F124010A7000224A70012219
:1021E000EDE711684FF0FF32E9E70000074B70B5EB
:1021F0000D467B4400F011F80446284600F020F814
:1022000010B14FF0FF3070BD204670BDC7FBFFFF1F
:1022100001694A1C02610878704700B58FB0CDE9AA
:1022200001310021059105497944CDE9031011469A
:102230006846FFF751FF0FB000BD0000E5FFFFFF4C
:10224000007B00F080007047754600F029F8AE462C
:1022500005006946534620F00700854618B020B5B2
:10226000FFF782FABDE820404FF000064FF000076C
:102270004FF000084FF0000B21F00701AC46ACE82E
:10228000C009ACE8C009ACE8C009ACE8C0098D469B
:1022900070470446AFF300802046FDF773FF00004F
:1022A0000048704780010020C8220008000000207C
:1022B00044000000280100080C230008440000200E
:1022C0009C0700004401000800A24A04000000002E
:1022D00000000000010203040607080900000000D6
:1022E00001020304010203040607080902040608A8
:1022F00000000000000000000000000000000000DE
:0C230000000000000000000000000000D1
:04000005080000ED02
:00000001FF
